:020000040800F2
:10000000203800200101000849120008410F0008B3
:1000100047120008610D0008F51E000800000000EE
:10002000000000000000000000000000351900087A
:100030009B0E00080000000025180008F9190008B0
:100040001B0100081B0100081B0100081B01000820
:100050001B0100081B0100081B0100081B01000810
:100060001B0100081B0100081B0100081B01000800
:100070001B0100081B0100081B0100081B010008F0
:100080001B0100081B0100081B0100081B010008E0
:100090001B0100081B0100081B0100081B010008D0
:1000A0001B0100081B0100081B0100081B010008C0
:1000B0001B0100081B0100084D1A00081B01000865
:1000C0001B0100081B0100081B0100081B010008A0
:1000D0001B0100081B010008C91C00081B010008C7
:1000E0001B0100081B0100081B010008DFF80CD0F1
:1000F00000F08EFB004800477129000820380020DE
:100100000648804706480047FEE7FEE7FEE7FEE7B1
:10011000FEE7FEE7FEE7FEE7FEE7FEE7FD19000863
:10012000ED00000830B505462A460B4612F8010BD3
:1001300013F8014B08B1A042F8D01CB1002802D03E
:100140006D1CF1E7284630BD421C10F8011B002948
:10015000FBD1801A704780EA010210B502F000431B
:10016000400022D04A001FD0010E01EB1261C0F303
:100170005600C2F3560240F4000042F40002A0FB15
:10018000022000047F39140400D0401C50EA1240C1
:1001900001D44000491EC2B20C0604EBD010401C32
:1001A0004008802A02D003E0002010BD20F00100AA
:1001B000002900DA0020184310BD30B480EA0102A3
:1001C00002F0004530F0004221F0004013D090B121
:1001D000C30DD40DC2F31601C0F31600E41A41F4A6
:1001E000000140F400027D34914201D3641C00E020
:1001F0004900002C02DA30BC002070474FF40000A8
:100200000023914201D3891A034340084FEA410178
:10021000F7D151B1914202D14FF0004105E002D235
:100220004FF0010101E06FF0010103EBC4502844DD
:1002300030BC00F0A1B896230022114600F0A5B80A
:100240000EB540F2334102910021CDE900110A467A
:100250000B4600F0D7F803B000BD00F0004220F0DC
:100260000040C10DC0F3160040F400007F2901DA00
:1002700000207047962903DCC1F19601C84001E0D7
:1002800096398840002AF4D04042704700F000427E
:1002900030F000400AD0C10D01F56071C0F31600C6
:1002A00042EA0151C208400711437047002001464D
:1002B000704701F0004330B421F0004150EA0102E0
:1002C00006D00A0DA2F56072C1F31301002A02DC08
:1002D00030BC00207047440F44EAC104C100E0185C
:1002E00030BC00EBC25000F047B830B50B460146B9
:1002F00000202022012409E021FA02F59D4205D3C5
:1003000003FA02F5491B04FA02F52844151EA2F16E
:100310000102F1DC30BD2DE9F05F05460020924678
:100320009B4688460646814640241BE028464146B7
:100330004746224600F08DFA53465A46C01A91416C
:1003400010D311461846224600F074FA2D1A67EBB6
:1003500001084F4622460120002100F06BFA17EBFE
:1003600000094E41201EA4F10104DFDC484631465D
:100370002A464346BDE8F09F0029A8BF7047401CAD
:10038000490008BF20F00100704710B4B0FA80FCAB
:1003900000FA0CF050EA010404BF10BC704749B1E8
:1003A000CCF1200421FA04F411FA0CF118BF012158
:1003B00021430843A3EB0C01CB1D4FEA00614FEA38
:1003C000102042BF002010BC704700EBC350104407
:1003D0000029A4BF10BC7047401C490008BF20F092
:1003E000010010BC704710B5141E73F1000408DA48
:1003F000401C41F1000192185B411A4301D120F0E9
:10040000010010BD2DE9F04D92469B4611B1B1FAA5
:1004100081F202E0B0FA80F22032904600F00AFA4F
:1004200004460F4640EA0A0041EA0B0153465A4689
:10043000084313D0114653EA010019D0C8F1400215
:10044000504600F006FA05460E46504659464246CA
:1004500000F0F0F9084305D0012004E020463946B9
:10046000BDE8F08D0020054346EAE0762C43374393
:100470000A986305E40AA0EB08000022FD0A44EA9A
:1004800047540A3002D500200146E9E7010510195A
:100490006941DDE9084500196941BDE8F04DA2E771
:1004A0002DE9FE4F804681EA0300C00F0C46009004
:1004B00021F0004123F00045B8EB0200A94105D22C
:1004C0004046214690461C460B46024623F000401B
:1004D000104347D0270DC7F30A00C3F30A51029017
:1004E000401A019040286BDAC3F3130040F4801BDC
:1004F0000098924620B10023D2EB030A63EB0B0B6A
:1005000001985946C0F14002504600F093F9064662
:100510000D4650465946019A00F0ABF910EB080021
:100520006141002487EA115284EAE7731A4340D0FC
:10053000009A62B3019A012A4FEA075215DC001BA8
:1005400061EB02014FF0004202EA0752CDE900429E
:10055000001C41F5801132462B46FFF753FF03B0D4
:10056000BDE8F08F40462146F9E7001B61EB020130
:10057000001C41F5801300185B412018A2F50017FC
:1005800047EB030140EAD570B6196D4111E06D08E3
:100590004FEA360645EAC0754FEA0752001B61EB89
:1005A0000201001C41F5801149084FEA3000001992
:1005B000514132462B4603B0BDE8F04FFFF713BF61
:1005C0000098012240000023D0EB020263EBE073AD
:1005D000009821464FEAE074B8EB000061EB04019B
:1005E000E9E783F000435BE781F0004158E72DE93C
:1005F000FE4F81EA030404F0004421F0004100941E
:100600004FF0000B23F0004350EA01045ED052EAA1
:1006100003045BD0C3F30A54C1F30A552C44A4F27B
:10062000F3340194A0FB0254C1F3130141F480118F
:10063000C3F3130343F4801301FB024400FB034E96
:10064000840A970A44EA815447EA8357A4FB07685F
:1006500002958D0A05FB07854FEA932C04FB0C5489
:100660002705029D4FEA065847EA1637B5EB0805FD
:100670006EEB070C870E920E47EA811742EA83124F
:10068000A7FB0201B6EB0B0164EB00042B0D43EA60
:100690000C335E1844EB1C50DA465146E7FB02016E
:1006A000C5F313044FEA0B3343EA14534FEA043201
:1006B000019C43EA0603A4F10C040294009CCDE9DA
:1006C00000B4FFF79FFE03B0BDE8F08F00200146A5
:1006D000F9E72DE9F04D81EA030404F0004B21F025
:1006E000004514464FF0000A23F0004150EA05028D
:1006F00020D054EA01021DD0C5F30A570246C5F3C3
:100700001303C1F31300C1F30A5640F4801543F4F8
:100710008013A7EB0608101BD64608F2FD3873EBD2
:10072000050002D308F1010801E092185B41B8F11D
:10073000000F03DA00200146BDE8F08D00204FF4E1
:100740008011064684460EE0171B73EB050705D3A0
:10075000121B63EB050306434CEA010C49084FEA00
:10076000300092185B4150EA0107EDD152EA0300D4
:1007700012D082EA040083EA0501084305D0101B69
:10078000AB4106D20122002306E000224FF00043D5
:1007900002E06FF0010253101AEB06004CEB085117
:1007A00010EB0A0041EB0B01BDE8F04DFFF71BBE5B
:1007B000C1F30A52C1F3130140F2FF3341F4801137
:1007C0009A4202DA00200146704740F233439A42CF
:1007D000A2F2334202DC524200F03BB800F02AB8E9
:1007E00030B5041E71F1000404DB4FF000444042B8
:1007F00064EB0101141E73F1000405DB1C464FF08D
:100800000043524263EB0403994208BF904230BD5B
:10081000064C074D06E0E06840F0010394E807004D
:1008200098471034AC42F6D3FFF764FCD45100086B
:10083000F4510008202A04DB203A00FA02F10020DB
:1008400070479140C2F1200320FA03F3194390400E
:100850007047202A04DB203A21FA02F00021704779
:1008600021FA02F3D040C2F1200291400843194618
:100870007047202A06DBCB17203A41FA02F043EA00
:10088000E07306E041FA02F3D040C2F12002914049
:1008900008431946704710B500F004F8BDE8104051
:1008A00000F0B2B8F8B50121042000F0E1FF4FF4E8
:1008B0000060ADF8000010240E4E8DF803400325B3
:1008C0008DF802506946304600F0E8FA0A490120E6
:1008D000C1F8AC01ADF8004028208DF803008DF878
:1008E00002506946304600F0D9FA4FF4E13002F088
:1008F000EFFCF8BD000801400000214270B504463D
:100900000D4610461946FFF7D4FC064620462946F8
:10091000FFF7CFFC314600F059F800F031F80C48F1
:10092000D0F8103100210B48012233B10378002B9D
:100930000DD10270417008A005E04378002B06D16C
:100940004270017009A0BDE8704001F0D5BA70BDD9
:10095000000021422E0000200D0A626C6520636FAA
:100960006E6E656374210D0A000000000D0A626C52
:100970006520646973636F6E6E656374210D0A0090
:100980002DE9F0410E4900240888020415D50D4FC9
:10099000C0F30E050020785508800B4E0BE0402177
:1009A000304601F00BFA0028F9D0395D304601F0ED
:1009B0009DFA641CA4B2AC42F1D3BDE8F081000002
:1009C0003000002010300020003801407CB5064681
:1009D0000846FFF75BFC04460D463046FFF756FC21
:1009E00002460B4602A0CDE9004502F055FC7CBD55
:1009F00057524A3A20252E316620626D7020252EEE
:100A000031662025252000007CB5654E0025C6F8FE
:100A1000A051644C0DE00A2263A165A001F022FF01
:100A200070B1D4F88801C043C4F88801642001F093
:100A300069FF052260A15EA001F014FF0028EAD141
:100A400005225FA15FA001F00DFF10B95EA001F0CB
:100A500053FA5FA260A1634801F05EFA0A2258A12E
:100A6000604801F0FFFE5F4900287DD05EA001F0E4
:100A700043FA60A262A15B4801F04EFA0A2250A13B
:100A8000584801F0EFFE5749002877D056A001F0F2
:100A900033FA06225DA1534801F03EFA0A2248A12A
:100AA000504801F0DFFE4F49002869D04EA001F008
:100AB00023FA0124CDE9005408234FF4E13256A172
:100AC000484801F029FA0A223DA1464801F0CAFE31
:100AD0004449002856D044A001F00EFA052253A143
:100AE000404801F019FA0A2235A13E4801F0BAFE49
:100AF0003C49002848D03CA001F0FEF90A2230A170
:100B00004EA001F0AFFE002840D051A001F0F4F952
:100B10000A222BA155A001F0A5FE002838D056A02E
:100B200001F0EAF90A2226A159A001F09BFE002853
:100B300030D05CA001F0E0F90A2221A161A001F00F
:100B400091FE002828D063A001F0D6F9532267A1B6
:100B5000244801F0E1F90A2219A1224801F082FE9D
:100B6000204900281AD001E006E007E01EA001F0AD
:100B7000C3F9C6F8A0417CBD5FA078E75EA086E718
:100B80005DA094E75CA0A7E75BA0B5E75DA0BDE72B
:100B900062A0C5E766A0CDE76CA0D5E756A0E6E762
:100BA00000002142008022424552524F5200000074
:100BB0002B2B2B6100000000612B6F6B00000000ED
:100BC0004F4B0000415400004154204F4B0D0A0090
:100BD00041544B2D57524A0041542B4E414D453DF7
:100BE00025730000D02B0020257320204552524F42
:100BF000520D0A0041544B2D57524A30310000002B
:100C000041542B48454C4C4F3D25730041542B54C7
:100C1000504C3D256400000041542B554152543D39
:100C200025642C25642C25642C25640041542B411B
:100C3000445054494D3D25640000000041542B4C64
:100C4000494E4B50415353454E3D4F4646000000E0
:100C500041542B4C494E4B50415353454E3D4F460A
:100C60004620204552524F520D0A000041542B4C51
:100C70004544454E3D4F4E0041542B4C4544454E56
:100C80003D4F4E20204552524F520D0A00000000A9
:100C900041542B534C415645534C454550454E3DD0
:100CA0004F46460041542B534C415645534C454505
:100CB00050454E3D4F464620204552524F520D0A58
:100CC0000000000041542B4D41585055543D4F46B3
:100CD0004600000041542B4D41585055543D4F465D
:100CE0004620204552524F520D0A000041542B4DD0
:100CF0004F44453D25630000257320204F4B0D0ACE
:100D00000000000041542B4C494E4B504153534579
:100D10004E3D4F464620204F4B0D0A0041542B4C70
:100D20004544454E3D4F4E20204F4B0D0A000000DC
:100D300041542B534C415645534C454550454E3D2F
:100D40004F464620204F4B0D0A00000041542B4DCA
:100D500041585055543D4F464620204F4B0D0A00F8
:100D6000FEE70029016802D041F0010102E04FF6E0
:100D7000FE7211400160704701684FF6FE7211402B
:100D800001600021016041608160C1603149314AE8
:100D90000839904203D1486840F00F0006E02D4A20
:100DA0001432904204D1486840F0F0004860704727
:100DB000284A2832904203D1486840F47060F5E731
:100DC000244A3C32904203D1486840F47040EDE739
:100DD000204A5032904203D1486840F47020E5E741
:100DE0001C4A6432904203D1486840F47000DDE749
:100DF000184A7832904203D1486840F07060D5E7D5
:100E0000154A111F904203D1086840F00F0006E018
:100E1000114A1432904204D1086840F0F000086092
:100E200070470D4A2832904203D1086840F4706040
:100E3000F5E7094A3C32904203D1086840F470401B
:100E4000EDE7054A50329042EAD1086840F470203C
:100E5000E5E70000080002400804024030B50268DF
:100E600047F6F0739A430C6A8B682343D1E9044533
:100E70002C4323438C692343CC6923434C6A23438B
:100E80008C6A234313430360CA6842600A68826025
:100E90004968C16030BD416070477047F0B5CC789B
:100EA000002204F00F03E40601D58C7823430C786C
:100EB0004FF00F0C14F0FF0F4FF0010E1BD0056820
:100EC0000E880EFA02F42640A64210D196000CFAC3
:100ED00006F725EA070703FA06F5CE783D43282EE4
:100EE00002D0482E02D002E0446100E00461521CAE
:100EF000082AE5D305600A88FF2A1CD94468002225
:100F000002F108060EFA06F50E882E40AE420ED10A
:100F100096000CFA06F7BC4303FA06F7CE783C437A
:100F2000282E00D14561CE78482E00D10561521C93
:100F3000082AE5D34460F0BD416170470161704704
:100F4000FEE70320401EC0B2FCD2704738B5012135
:100F5000102000F08DFC10208DF803004402ADF845
:100F600000400320054D8DF8020069462846FFF732
:100F700095FF21462846FFF7DFFF38BD00100140EE
:100F800070B5094C0025C4F8A85104F5D47400F0DC
:100F900081F86560022001F0C9FC01202060022078
:100FA00001F0C4FC256070BD0080214208B501211C
:100FB000082000F05DFC4FF44060ADF80000102008
:100FC0008DF8030003208DF8020069460448FFF7FE
:100FD00065FF04480121C0F8A811C0F8AC1108BD94
:100FE000000C01400080214270B5094C0026C4F875
:100FF000A86104F5D47400F04DF801256560022065
:1010000001F094FC2560022001F090FC266070BD88
:10101000008021422DE9F0478146002400F028F8A5
:101020000025124E2F464FF00108C6F8A871022085
:1010300001F07CFCC6F8A8816006040ED6F82C01ED
:1010400008B1641CE4B2012001F070FC6D1CEDB22B
:10105000082DEAD3B9F1000F04D0FFF791FF204625
:10106000BDE8F087FFF7C0FFF9E7000000802142EC
:1010700008B54FF40060ADF8000003208DF80200C1
:1010800048208DF8030069460148FFF707FF08BDB7
:10109000000C014008B54FF40060ADF800000320DB
:1010A0008DF8020010208DF8030069460148FFF713
:1010B000F5FE08BD000C01402DE9F0410546FFF7A3
:1010C000E9FF0F4E0027C6F8A8713C464FF0010813
:1010D000E809C6F8AC016806050E022001F026FCFE
:1010E000C6F8A881022001F021FCC6F8A8710220F0
:1010F00001F01CFC641CE4B2082CE9D3BDE8F081CB
:101100000080214270B5FFF7C5FF094C0120C4F8EB
:10111000AC01C4F8A801042004F5D47401F006FC65
:1011200000256560042001F001FC256070BD000011
:101130000080214210B5FFF7ADFF094C0020C4F834
:10114000A801C4F8AC01042004F5D47401F0EEFB4E
:10115000012020606060BDE81040042001F0E6BB83
:101160000080214270B50024FFF782FF0D4D01265B
:10117000C5F8AC61304601F0D9FBC5F8A861012083
:1011800001F0D4FB07E0641CE4B2FA2C03D9FFF7AA
:10119000D1FF012070BDD5F82C010028F3D1C5F88E
:1011A000A80170BD0080214208B50121082000F08F
:1011B0005FFB4FF48040ADF8000048208DF803003D
:1011C00069461A48FFF76AFEFFF7F0FE00F030F8B4
:1011D000C021022001F08EFD0021032001F08AFDD4
:1011E0000021042001F086FD0021052001F082FD90
:1011F0000021062001F07EFD0F21082001F07AFD7C
:101200000321092001F076FD27210A2001F072FD5B
:1012100024210C2001F06EFD24210D2001F06AFD37
:101220007F21102001F066FD08BD0000000C014088
:1012300010B54021092001F05DFD4021BDE81040BE
:10124000092001F057BDFEE77047000030B50F23BD
:10125000C27801780125F2B1144A126801F1E02147
:1012600002F4E062C2F5E062120AC2F10404D34063
:101270004278A24084781C401443220181F8002463
:10128000007800F01F018D404009800000F1E0204F
:10129000C0F8005130BD01F01F00854048098000B2
:1012A00000F1E020C0F8805130BD00000CED00E0FE
:1012B00030B40021084B0A46002003EBC004401C58
:1012C000C0B262548028F8D3491CC9B20829F3D3AC
:1012D00030BC00F005B90000F00F002030B5CC089C
:1012E00001F0070301259D40EBB2064D05EBC0055B
:1012F000C808285C0AB1184302E063EA0000C04352
:10130000285530BDF00F002070B50E4D4FF400741D
:1013100021462846FFF712FE661031462846FFF7A1
:101320000DFEFFF70EFE21462846FFF705FEFFF7EC
:1013300008FE31462846FFF7FFFDBDE87040FFF785
:1013400000BE0000000C014070B5094D4FF4007460
:1013500021462846FFF7F0FD61102846FFF7EEFD15
:10136000FFF7EFFD21462846BDE87040FFF7E6BDD8
:10137000000C014070B50B4C4FF400712046FFF794
:10138000DDFDFFF7DEFDA51529462046FFF7D6FD5A
:10139000FFF7D7FD29462046FFF7CEFDBDE8704098
:1013A000FFF7CFBD000C014038B50121082000F047
:1013B0005FFA4FF48074ADF8004014208DF80300FC
:1013C0000320424D8DF8020069462846FFF766FD6E
:1013D00021462846FFF7B2FD6400ADF8004069469B
:1013E0002846FFF75BFD21462846FFF7A7FDC820EA
:1013F00001F088FA0021AE2000F0F9F9002108463A
:1014000000F0F5F90021102000F0F1F90021402052
:1014100000F0EDF90021812000F0E9F90021CF2052
:1014200000F0E5F90021A12000F0E1F90021C82039
:1014300000F0DDF90021A62000F0D9F90021A82054
:1014400000F0D5F900213F2000F0D1F90021D32090
:1014500000F0CDF90021084600F0C9F90021D5209F
:1014600000F0C5F90021802000F0C1F90021D92049
:1014700000F0BDF90021F12000F0B9F90021DA20D7
:1014800000F0B5F90021122000F0B1F90021DB20B5
:1014900000F0ADF90021302000F0A9F90021202052
:1014A00000F0A5F90021022000F0A1F900218D2013
:1014B00000F09DF90021142000F099F9FFF7F8FEE3
:1014C0000021AF2000F093F938BD0000000C01406E
:1014D0000346012000E05843491EC9B2FBD27047C1
:1014E00070B5174E002505F1B000C0B2002100F024
:1014F0007EF90021084600F07AF90021102000F062
:1015000076F9FFF701FF782000F01CF8FFF732FFB3
:10151000402000F017F8FFF72DFF002406EBC40071
:10152000405D00F00FF8FFF725FF641CE4B2802C4B
:10153000F4D3FFF709FF6D1CEDB2082DD3D370BDB6
:10154000F00F00202DE9F041114F002405464FF423
:101550000078BE1528064146384602D5FFF7EEFC56
:1015600001E0FFF7E9FCFFF7ECFC31463846FFF7F6
:10157000E5FCFFF7E6FC31463846FFF7DDFC680680
:10158000641C050EE4B2082CE4D3BDE8F081000031
:10159000000C01402DE9FC5F1D46884681468B46C4
:1015A0000090082B0DD0680700D0012000EBD5007B
:1015B00069084843C0B2203A02F0FF0A00260190B1
:1015C00046E00620F7E7082D10D00C2D14D0102D82
:1015D00016D0182D45D124490AEBCA0001EB800032
:1015E0000027845DE0070FD00C9A10E01F490AEB3A
:1015F0004A0001EB4000F3E70AEB4A001C49EDE723
:101600001C4901EB0A10EBE70C9840B3002241465D
:101610004846FFF763FE7F1C640808F10100FFB233
:1016200000F0FF08082FDDD309F1010000F0FF09E9
:10163000082D0AD00099A9EB0100B0EB550F04D199
:101640000BF10800894600F0FF0B761CD846F6B275
:1016500001988642B7D3BDE8FC5FFFF741BF012286
:10166000D5E7BDE8FC9F000038400008AC33000817
:10167000D4350008483A00082DE9FC5F8146009007
:101680001E46924688468B46580700D0012000EB44
:10169000D60070430025019041E0102E0ED0182E88
:1016A00010D0202E15D0402E42D1224901EB4A20E5
:1016B0000027445DE00711D00C9A12E01E4901EBAF
:1016C0004A10F5E71C490AEBCA00803101EBC00063
:1016D000EEE71849803901EBCA10E9E70C9828B306
:1016E000002241464846FFF7F9FD7F1C640808F1D7
:1016F0000100FFB200F0FF08082FDBD309F1010061
:10170000009900F0FF09A9EB0100B04204D10BF1F0
:101710000800894600F0FF0B6D1CD846ADB2019859
:101720008542BAD3BDE8FC5FFFF7DABE0122D8E7F5
:10173000BDE8FC9FDC4E0008944D00082DE9F84FF1
:101740000025DDE90A691F4692468B468046082E31
:1017500000D1022500241CE0381B401EC1B20A2023
:10176000FFF7B6FEBAFBF0F00A21B0FBF1F201FB85
:101770001200CDF8009090B13030C2B205EB5601A6
:1017800001FB0480C0B233465946FFF703FF641CD7
:10179000E4B2BC42E0D3BDE8F84FFFF7A1BE05EBD1
:1017A000560101FB0480C0B233463022ECE72DE93C
:1017B000F8431E46154688460446089F0BE033460C
:1017C000414620460097FFF7E5FE082E0CD004EBBB
:1017D0005600C4B26D1C2A78A2F120005E28EED912
:1017E000BDE8F843FFF77CBEA41DE4B2F2E770B594
:1017F0000C460546FFF788FD7820FFF7A3FEFFF7AC
:10180000B9FD0CB1402000E00020FFF79BFEFFF780
:10181000B1FD2846FFF796FEFFF7ACFDBDE870402E
:10182000FFF792BD70470000044A0029516901D0BA
:10183000014300E081435161704700000010024005
:10184000044A0029D16901D0014300E08143D161FC
:101850007047000000100240044A0029116901D0BD
:10186000014300E081431161704700000010024015
:10187000044A0029916901D0014300E0814391614C
:101880007047000000100240044A0029D16801D0CE
:10189000014300E08143D160704700000010024026
:1018A00030B5204A5168204B11F00C0103D00429B7
:1018B00001D0082901D0036012E05168536801F497
:1018C00070114FF0020413F4803F04EB914102D0F9
:1018D00053689B0301D5154B00E0134B594301603E
:1018E00051680F2303EA1111114B5C5C0168E14060
:1018F00041605468072505EA14241C5D21FA04F4AC
:101900008460546805EAD4241B5DD940C1605268E4
:10191000032303EA9232064B1B1F9A5CB1FBF2F1E0
:10192000016130BD0010024000127A0000093D0044
:101930003A000020704700000CB5002226480092B3
:101940000192016841F4803101604FF4A0630168A5
:1019500001F4003101910099491C0091019911B9DC
:1019600000999942F3D10168890333D5012101918E
:101970001A490A6842F010020A600A6822F003025B
:101980000A600A6842F002020A60416841604168E8
:101990004160416841F480614160416821F47C11FB
:1019A0004160416841F4E8114160016841F0807193
:1019B000016001688901FCD5416821F003014160A3
:1019C000416841F0020141604168C1F3810102298F
:1019D000FAD10CBD01920CBD001002400020024063
:1019E0004FF0E0210428086903D020F004000861CA
:1019F000704740F00400FAE7704700000F4810B548
:101A0000016841F00101016041680D4A11404160E7
:101A100001680C4A11400160016821F480210160D5
:101A2000416821F4FE0141604FF41F018160FFF71E
:101A300083FF05494FF00060086010BD00100240B0
:101A40000000FFF8FFFFF6FE08ED00E010B50B4CBC
:101A50000121204600F063F800280DD00121204626
:101A600000F050F80648018841F400410180BDE8CB
:101A70001040002000F032B810BD00000008004007
:101A8000300000207FB50D46044601210420FFF7F9
:101A9000D7FEADF804400020ADF800500E4CADF874
:101AA0000600ADF802006946204600F04FF801221A
:101AB0001146204600F03FF81E208DF80C00012052
:101AC0008DF80D0002218DF80E108DF80F0003A87F
:101AD000FFF7BCFB7FBD00000008004010B5084ABE
:101AE0004FF0000130B11446104600F02CF80121EF
:101AF000204600E01046BDE8104000F006B80000A7
:101B000000080040C943018270470029018802D0C3
:101B100041F0010101E021F001010180704702461E
:101B20000020138A92890B4202EA010202D0002AA5
:101B300000D001207047002A828901D00A4300E0CA
:101B40008A438281704781847047000030B50288E3
:101B50001B4C1C4DA0420DD0A8420BD0B0F1804FC1
:101B600008D0194B984205D0184B984202D0184B18
:101B7000984203D122F070034A881A43154B9842C9
:101B800006D0154B984203D022F44073CA881A43FA
:101B900002808A8882850A880285A0420AD0A842EB
:101BA00008D00E4A904205D00D4A904202D00D4A0C
:101BB000904201D1097A01860121818230BD000065
:101BC000002C0140003401400004004000080040A7
:101BD000000C004000100040001400400040014094
:101BE000004401400048014070B50C460646012102
:101BF0008CB015460846FFF717FE3046FFF7BCF8D5
:101C000000211020CDE902018020CDE9041040011F
:101C1000CDE9081006910A91079169463046CDE951
:101C20000045FFF71BF90CB070BD70B50C460546BA
:101C30000021FFF796F821462846FFF72CF92846A1
:101C4000BDE870400121FFF78CB8000010B586B0E8
:101C5000012144F20400FFF70BFE4FF40070ADF8D1
:101C6000100018208DF813000320154C8DF8120079
:101C700004A92046FFF712F92115ADF81010042130
:101C80008DF8131004A92046FFF708F94FF4E1304E
:101C900000900020ADF80400ADF80600ADF8080093
:101CA000ADF80C000C20074CADF80A006946204640
:101CB00000F0C2F80121204600F034F806B010BD53
:101CC000000801400038014070B5124C40F2255127
:101CD000204600F07AF8002818D0204600F002F9DB
:101CE0000D4DC4B22888010410D4B0F5806F0ED217
:101CF00000210A48FFF727FF288810B90120FFF7C5
:101D0000EDFE074928880C54401C288070BD40F423
:101D10000040FAE700440040300000200008004086
:101D2000103000200029818902D041F4005101E0E7
:101D300021F4005181817047002A828A01D00A4330
:101D400000E08A4382827047174910B588420AD161
:101D500001218C032046FFF797FD2046BDE8104087
:101D60000021FFF791BD1149884202D101214C04A5
:101D700010E00F49884202D101218C040AE00D498C
:101D8000884202D10121CC0404E00B4988420AD1E7
:101D900001210C052046FFF75FFD2046BDE81040FD
:101DA0000021FFF759BD10BD00380140004400403C
:101DB00000480040004C0040005000400246002017
:101DC00012880A4200D00120704770B501F01F054B
:101DD00001260024C1F3421306FA05F2012B0FD0AD
:101DE000022B0FD0838A4FEA11210088134206FA92
:101DF00001F600EA060001D000B10124204670BDC2
:101E00008389F0E7038AEEE710B5C1F3421301F0CE
:101E10001F040121A140012B07D0022B07D0143051
:101E2000002A026805D00A4304E00C30F8E71030BD
:101E3000F6E78A43026010BD30B50446008A85B0DB
:101E40000D464CF6FF710840E98801432182A089C4
:101E50004EF6F3110840A9882A8911436A89024382
:101E60001143A181A08A4FF6FF410840A98901438F
:101E7000A1826846FFF714FD1948844201D10398F6
:101E800000E00298A189090400EBC00101EB0010F9
:101E9000296801D5490000E08900B0FBF1F0642217
:101EA000B0FBF2F109010B096FF018056B4300EB71
:101EB0008300A3891D044FF0320306D503EBC00055
:101EC000B0FBF2F000F0070005E003EB0010B0FB00
:101ED000F2F000F00F000843208105B030BD000093
:101EE000003801408088C0F308007047C1F3080142
:101EF00081807047FEE700000FB4054B10B503A9C1
:101F0000044A029800F000F910BC5DF814FB0000D0
:101F1000552900084C0000200FB4084B10B504A947
:101F200002AA039800F0F0F8044602A9002000F08D
:101F300082FC204610BC5DF814FB00003728000826
:101F400037B514460846064B6A46214600F0DCF8D1
:101F500004466946002000F06EFC20463EBD0000AD
:101F60003728000802E008C8121F08C1002AFAD169
:101F700070477047002001E001C1121F002AFBD109
:101F8000704700002DE9FF5F82B00021DDE90430D9
:101F9000020DDDF840B0034318D044F61050A2F211
:101FA000FF3242431514119801281FD0A5EB0B00F6
:101FB000401C5FEA000A4FF000064E4FDFF83891F0
:101FC000B046504615D5CAF1000413E0119801241B
:101FD0004AA3012801D16FEA0B010298119AC0E9C6
:101FE0000031C0E9024206B0BDE8F09FCBF100002D
:101FF000DFE704460021404A491842EB0450CDE98E
:10200000001012E0E00707D032463B464046494602
:10201000FEF7EDFA8046894632463B4610461946A1
:10202000FEF7E5FA06460F466410002CEAD1DDE91A
:102030000401DDE90023BAF1000F06DAFEF7D7FA52
:1020400042464B46FEF7D3FA05E0FEF742FB424616
:102050004B46FEF73EFB04460E460022284BFEF799
:10206000BFFB03D84FF0FF30014607E00022254BAD
:1020700020463146FEF714FAFEF79AFB102409E0D9
:10208000002C0ADB0A220023FEF745F9039B3032BD
:102090001A55641E50EA0102F2D1641C039AC4F17D
:1020A00011031444119A012A03D0012208430DD1CF
:1020B0000AE0084304D000204FF0110B119072E7A2
:1020C000A3EB0B056D1E0DE05B4504DD4FF0000238
:1020D00005F1010504E003DA4FF00002A5F1010566
:1020E000002AECD002981199C0E90231C0E90045FC
:1020F00079E70000000014400000F03F30000000CD
:102100000000F0430000E03F2DE9FF4F95B09B46F3
:102110008946064600250FE2252877D10024274668
:10212000F84A0121059400E0044316F8013F203BE2
:1021300001FA03F01042F7D130782A2811D06FF05D
:102140002F033078A0F13002092A16D8059A44F0FE
:10215000020402EB820203EB42021044761C05905B
:10216000EFE759F8042B0592002A03DA504244F4B1
:102170000054059044F00204761C30782E2816D1C5
:1021800016F8010F44F004042A280DD06FF02F0236
:102190003078A0F13003092B09D807EB870302EB55
:1021A0004303C718761CF3E759F8047B761C307894
:1021B0006C280FD006DC4C2817D068280DD06A2870
:1021C00014D104E0742810D07A280FD10DE044F423
:1021D00000140AE044F4801401E044F440147278DE
:1021E000824202D104F58014761C761C3078662871
:1021F0000BD013DC582877D009DC002875D045288F
:10220000F6D04628F4D047281AD19DE118E063287B
:1022100035D0642879D0652812D195E1702873D023
:1022200008DC6728F1D069286FD06E280DD06F28A0
:1022300006D1B5E073282CD0752875D0782874D0D5
:102240005A46179990476D1C75E1C4F30250022855
:1022500009D003280DD0D9F8001004280DD00D6046
:1022600009F1040967E1D9F80010EA17C1E9005241
:10227000F6E7D9F800100D80F2E70D70F0E719F8D5
:10228000041B8DF8001000208DF80100EA460120A3
:1022900003E059F804AB4FF0FF3061074FF0000145
:1022A00002D40DE008F101018846B9420FDA8045F9
:1022B000F8DB1AF808100029F4D108E008F1010150
:1022C00088468142FADB1AF808100029F6D10598F1
:1022D0005B46A0EB080721463846179A00F094FAAF
:1022E000284400EB080507E04DE029E10DE01AF86D
:1022F000010B5A4617999047B8F10108F7D25B468F
:1023000021463846179A13E142E00A220092C4F3AC
:1023100002524FF0000A022A08D059F804CB032ACF
:102320004FEAEC710AD00DE029E02AE009F107013B
:1023300021F00702F2E802C1914609E00FFA8CFC95
:102340004FEAEC71042A03D14FFA8CFC4FEAEC718E
:10235000002907DA0A460021DCF1000C61EB0201DA
:102360002D2202E0220504D52B228DF80420012223
:1023700003E0E20701D02022F7E7904659E00A2166
:1023800002E010220DE010214FF0000A00910BE056
:1023900010224FF0000A44F004040827009203E0E2
:1023A00008224FF0000A0092C4F30252022A05D01C
:1023B00059F804CB0021032A08D009E009F10701EC
:1023C00021F00702F2E802C1914605E01FFA8CFCF9
:1023D000042A01D10CF0FF0C4FF00008220728D589
:1023E000702806D0009B83F0100353EA0A0305D03F
:1023F0000EE040228DF80420012208E05CEA010290
:1024000006D030228DF804208DF805000222904677
:10241000009B83F0080353EA0A030AD15CEA010235
:1024200001D1620705D530228DF804204FF0010854
:102430007F1E582804D034A003900EA802900DE00F
:1024400036A0F9E753466046009AFDF764FF8446DC
:102450000398825C0298401E029002705CEA0100C0
:10246000F0D1029806A9081A00F1200A600702D5E7
:1024700024F4803400E00127574502DDA7EB0A0071
:1024800000E0002000EB0A01009005984144401A4A
:102490000590E00306D45B462146179A059800F0A4
:1024A000B3F90544002706E001A85A46C05D179914
:1024B00090476D1C7F1C4745F6DBE0030CD55B465F
:1024C0002146179A059800F09FF9054404E0302052
:1024D0005A46179990476D1C0099481E0090002994
:1024E000F5DC08E0029802995A460078491C0291EE
:1024F000179990476D1CBAF10001AAF1010AF1DCAD
:1025000065E10000092801003031323334353637B7
:10251000383961626364656600000000303132332F
:1025200034353637383941424344454600000000CF
:1025300000F058F90544761C307800287FF4ECADA3
:1025400019B02846BDE8F08F620700D4062709F1CC
:10255000070222F0070CFCE80223E14603F00048E2
:102560005FEA080C02D00FF2702C0DE05FEA045C09
:1025700002D50FF2682C07E05FEAC47C02D00FF2AC
:10258000602C01E0AFF2700C4FF0FF3823F00043F5
:10259000CDF850C065280CD006DC452809D0462867
:1025A0001DD047283DD13DE0662818D067287ED150
:1025B00038E00021112F01DB112000E0781CCDE96B
:1025C000000106A90EA8FFF7DDFCDDE90F010E9A58
:1025D00003910021009207F1010A04914DE04FF0B0
:1025E00000400097CDE9011006A90EA8FFF7CAFC2C
:1025F000DDE90F0203920E9B11990022DDF80CA079
:102600000093049211B9791C00EB010AB7EB0A00A0
:1026100004D4C0F1FF3007F1010A0490AAEB0700CF
:10262000019044E0012F00DA01270021112F01DD84
:10263000112000E03846CDE9000106A90EA8FFF7F9
:10264000A1FCDDE90F010E9A039100210491009293
:10265000BA4621070CD40399514500DA8A46BAF1EB
:10266000010F05DD009AAAF10101515C302908D063
:10267000B84202DA10F1040F06DA0121CDE90110A7
:1026800015E0AAF10101E9E7002805DC04990144FD
:102690000491AAEB000102E0411C514500DD8A468D
:1026A0000499401A401C01904FF00040029020070E
:1026B00004D40198504501DBCDF8048000208DF84A
:1026C0004F0002980DF14F07B0F1004F25D02B209D
:1026D0000E9002984FF0020800280CDA4042029057
:1026E0002D200E9007E00A210298FDF7FEFD303103
:1026F000029007F8011DB8F10001A8F10108F2DC11
:1027000002980028EFD1791E0E980870307800F0FA
:10271000200040F0450007F8020D12A8C01B00F190
:1027200007081498007800B1012000EB0A01019815
:1027300001EBE07105984144401A401E0590E0030A
:1027400006D45B462146179A059800F05DF80544CB
:102750001498007818B15A46179990476D1CE003F9
:1027600024D55B462146179A059800F04DF805449C
:102770001CE00498002807DBDDE90301884203DD43
:102780000098405C179901E0179930205A4690470D
:10279000049805F10105401C04900198401E019029
:1027A00004D12E205A46179990476D1CBAF10001AA
:1027B000AAF1010ADDDC05E017F8010B5A4617996A
:1027C00090476D1CB8F10001A8F10108F4DC5B46EC
:1027D0002146179A0598ABE62D0000002B0000005B
:1027E000200000002DE9F041044600251E46174652
:1027F000880404D405E039462020B0476D1C641ECF
:10280000F9D52846BDE8F0812DE9F04104460025C0
:102810001E469046C80301D5302700E020278804D3
:1028200004D505E041463846B0476D1C641EF9D515
:102830002846BDE8F0810A68531C0B601070704791
:10284000064A014600201288130406D5044BC2F341
:102850000E0298541846FDF765BC70473000002002
:10286000103000202DE9F0410027164D884614460F
:1028700001463E462F80FF2807D81348D0F8842011
:10288000002AFBD11148018002E011A000F004FDF4
:10289000B8F1000F13D06CB911E00A2000F032F843
:1028A0002888000406D54046FFF7CAFF2E8008B1ED
:1028B00024B104E0641E2404240CEED10127384620
:1028C000BDE8F081300000200000024004440040D8
:1028D00025730D0A0000000010B504466FF00400D7
:1028E000FFF77EF80649E00800EB40020870C2EBF3
:1028F000C0104FF6FF7202EAC000488010BD000011
:10290000320000200849498848434FF0E0214861DF
:1029100000238B61012008610869C20701D0C00350
:10292000FAD50B618B6170473200002008490978A5
:1029300048434FF0E021486100238B61012008618A
:102940000869C20701D0C003FAD50B618B617047DB
:102950003200002070B5054C0546C1B22046FFF795
:10296000C5FA20880006FCD5284670BD0038014015
:102970000EB54820FFF7B0FFFEF7E8FAFEF714FDAA
:102980003220FFF7BFFFFEF793FCFEF70DFCFFF7C9
:102990005DF9FDF780FFDFF8D8824FF0000B454668
:1029A000B248C5E9040B4FF0010A5E4654461023B5
:1029B0005A4659465846CDF800A0FEF75DFE102352
:1029C0000122002118460094FEF756FE10233A22F9
:1029D000002128200094FEF7DDFD1023A5A2002190
:1029E00050200094FEF7E3FE102302221946002037
:1029F0000094FEF741FE1023032219461846009466
:102A0000FEF73AFE10233A22194628200094FEF7DA
:102A1000C1FD10232522194650200094FEF7BAFD6F
:102A20004FF4FA70944CEE61686008F1280904F5DF
:102A3000FA659248D0F81C010128FAD08C49072089
:102A4000283100F076F999F8000099F80120800704
:102A5000800B40EA022099F80220D8F81C3010437D
:102A6000424645F8230099F8036099F80470B607C8
:102A7000B60B99F8051046EA07260E4344F8236082
:102A8000D8F81010884200D210615169884200D9EC
:102A900050615B1CD361D8F804008342C9DB55F850
:102AA00023009061724AD21C501E02F109018DE888
:102AB0000700831D724A7048D8F8041000F090F99E
:102AC0004FF4FA786A4A64206D4DD06105EB8003BB
:102AD000A3F5805355F8201004EB8006C3F8701E50
:102AE000A6F5805654F82030C6F8703E1369994216
:102AF00000D211615369994200D95161401CD061E3
:102B00004045E3DB4FF4C8701546D0615C4FE8697F
:102B100007EB800050F8040CA8615848D0F81C114D
:102B20000129FBD052490720283100F002F999F819
:102B3000000099F801208007800B40EA022099F8F4
:102B40000220EE69104347F8260099F8032099F80F
:102B500004309207920B99F8051042EA03220A43C7
:102B600044F82620A969884219D9401AFDF763FB69
:102B70000746D5E90410401AFDF75DFB01463846CB
:102B8000FDF71BFB3F49FDF7E6FA6862FDF765FBC1
:102B9000296A081A28621CD5C5F820B019E0081A5D
:102BA000FDF749FB0746D5E90410401AFDF743FB42
:102BB00001463846FDF701FB3249FDF7CCFA686261
:102BC000FDF74BFB296A08442862FF2801DDFF203E
:102BD0002862E878012805D1E868782802DA2870A8
:102BE000287A02E0584685F800B0761C6870EE61DD
:102BF00046458BDB1E4AD21C501E02F109018DE8AE
:102C00000700831D1E4A1C48696800F0E9F82A780D
:102C10004FF010014FF003030AB3CDE9001A002171
:102C20002F20143AFEF78AFD1020CDE9000A014654
:102C300002236A782F20FEF781FD6A78297812A096
:102C4000FFF75AF96878FDF7FBFA06460F46287831
:102C5000FDF7F6FA32463B46FDF750FE32E7CDE986
:102C6000001A002211462F20DCE70000FFFF0300BE
:102C700000000020424D5000500000200000214282
:102C80002008002000007F43E5BF83E78E873D20BA
:102C900025642042504D20E8A180E6B0A73D2025C4
:102CA000640D0A200000000010B50446FEF72AFA61
:102CB000AE20FEF701FAFEF755FA68B92046FEF796
:102CC000FBF9FEF74FFA38B9FEF71CFAAF20FEF712
:102CD000F3F9FEF747FA18B1FEF72CFA002010BD01
:102CE0000020FEF797F90446FEF77EF9FEF722FA78
:102CF000204610BD70B50C460546FEF703FAAE201F
:102D0000FEF7DAF9FEF72EFA58B92846FEF7D4F99D
:102D1000FEF728FA28B92046FEF7CEF9FEF722FA88
:102D200018B1FEF707FA002070BDFEF703FA012084
:102D300070BD70B505460C460020FFF7B5FF0120B9
:102D4000FFF7B2FFFEF7DEF9AE20FEF7B5F9FEF7AA
:102D500009FA38BB2846FEF7AFF9FEF703FA08BBBD
:102D6000FEF7D0F9AF20FEF7A7F9FEF7FBF9C8B9D7
:102D70000120FEF74FF920700120FEF74BF960703B
:102D80000120FEF747F9A0700120FEF743F9E0703B
:102D90000120FEF73FF920710020FEF73BF960713A
:102DA000FEF7C8F9BDE87040FEF7C4B92DE9F84157
:102DB0008046DDE90706009017460C46099D40460F
:102DC00000F0D0F933463A462146404600F0FDF97E
:102DD0002068A84200DB28462060BDE8F88100009A
:102DE0002DE9FF4FB6B00C46DDE9449506460021BB
:102DF0009246084603E056F82020401C1144A042A9
:102E0000F9DBB1FBF4F10020D14A05E056F820309F
:102E10005B1A42F82030401CA042F7DB002002EB96
:102E2000800152F820304F683B44D1E902713944A7
:102E30001944CB1701EB9371891042F82010401C04
:102E4000B0F5F87FEBDBC34900204FF4F773C04ABD
:102E500002EB800752F820C07F68A7EB0C0741F80F
:102E60002070401C9842F2DD002001EB800751F8F1
:102E700020207F689E463A4402EBD272521041F8FD
:102E80002020401C7045F0DBDFF8CCC200208B46D0
:102E900000210246471D08E0A2EB00085BF8223043
:102EA0003CF81880521C03FB1811BA42F4DB40F2C4
:102EB0007A4291FBF2F14BF82010401C5B46B0F5D2
:102EC000F47FE5DD00221046774653F820100029F4
:102ED00000DC4942B846401C0A444045F5DD40F25A
:102EE000EF1392FBF3F00822CDE9000205210291D5
:102EF000984A35A912A8FFF759FF359A00210DF11C
:102F0000480C022A1CDB012008E00CEB80075CF86F
:102F1000203057F8047CDB1B1944401C9042F4DB42
:102F2000521E91FBF2F041F2707191FBF0F0C9F882
:102F300000000120287000200DF1980E359B0AE05A
:102F40008648C9F800000020F4E75CF82010891CCE
:102F50004EF82010401C9842F7DB0020DFF8F0917B
:102F600009E056F820207E4949F820205AF8202010
:102F700041F82020401CA042F3DB002631461DE032
:102F80005EF821000122170600F1050CC44514DC8F
:102F9000441F002C11DD0DF10C0B401F09E059F806
:102FA0002040BC4204DA02B1002227464BF821003F
:102FB000401C6045F3DB02B9761C491C9942DFDBFB
:102FC000022E04DA3999654808600020BAE0002032
:102FD0004FF4F87C09EB800159F820404F68604AB3
:102FE0003C44D1E9027139442144CC1701EB94717E
:102FF000891049F8201002EB800152F820304C680B
:10300000CB462344D1E9024121441944CB1701EBBB
:103010009371891042F82010401C6045DADB0024CF
:10302000204621AA002142F82010401C0528F8DB88
:1030300000204FF4FA7205E003A951F820109142E4
:10304000C0DC401CB042F7DB0021761E009655E044
:1030500003A800EB81024FF07F46576850F821200B
:103060003346A7EB0208B8F10A0F46DD1046DFF839
:10307000F0900CE05BF820C09C4501DD6346824681
:1030800059F820C0B44501DD66460546401C87421C
:10309000F0DC59F827C059F822E05BF82770ACEB58
:1030A0000E00A5EB020C00FB0CF090FBF8FCE644D4
:1030B0005BF8220059F825C08146381AAAEB0202B3
:1030C000504390FBF8F202EB09005BF82520ACEBD3
:1030D0000E0E121A0EFB03F07243C011D211002A19
:1030E0000BDD052C09DA40B100EB8000800090FB7D
:1030F000F2F221A840F82420641C491C0098814267
:10310000A6DB214621A800F093F804EBD470401010
:10311000012821A90ADD01EB800251F8200052F8B4
:10312000042C104400EBD070401001E051F8200056
:10313000C11EB529BFF446AF07493E31085C399935
:1031400008600120439908703AB0BDE8F08F000094
:10315000301C002070140020DC50000819FCFFFF18
:10316000002400202DE9F04301240025DDF81C9007
:10317000A3F1010C0D6024E052F824704F451FDDCF
:1031800002EB840555F8045CAF4219DD012500E02F
:103190006D1C66199E4203DA52F826804745F7D027
:1031A000254452F82550AF4208DD0D680F2D05DA91
:1031B000AF006D1C0D60C451741C02E0344600E089
:1031C000641C6445D8DBBDE8F0832DE9F0431E465E
:1031D00013460C460A6805460146184600F040F8BA
:1031E0004FF0FF39484619E08C46411CC6F10008F3
:1031F000216010E055F82130421C17D055F82020EE
:103200009A1AB24201DC424504DA22689700521C45
:103210002260EB51491C6145ECDB401C2168814276
:10322000E2DC2846BDE8F04300F002B84A46E7E792
:1032300030B5012311E050F823501A4602E040F85F
:103240002240521E002A05DD00EB820454F8044C93
:10325000AC42F4DC40F822505B1C8B42EBDB30BD0F
:10326000F0B5012415E051F82460234602E041F84E
:1032700023505B1E002B09DD01EB830550F82670FF
:1032800055F8045C50F825C06745F0DC41F8236030
:10329000641C9442E7DBF0BD0FB40B4810B503AAE1
:1032A0000299FEF74DFE0948D0F884100029FBD1A1
:1032B0000548FCF749FF81B204488030FEF7B5FCB1
:1032C00010BC5DF814FB0000102C00200000024030
:1032D0002DE9FC41044601210420FEF7C9FA012131
:1032E0004804FEF7ADFA2B4E3046FEF72DFD0420C4
:1032F000ADF8000003258DF802501820264F8DF8F8
:10330000030069463846FDF7C9FD0820ADF8000006
:1033100048208DF8030069463846FDF7BFFD1F4978
:103320000C200C6000248C80CC800C818C81488126
:103330003046FEF781FD012280213046FEF7FCFC7D
:10334000174A311D1748FEF74FFC01213046FEF7A2
:10335000E9FC012240F225513046FEF755FD2620BA
:103360008DF8040002208DF805008DF8065001202C
:103370008DF8070001A8FDF769FF41F61F416320A2
:10338000FEF780FB084804800020FEF7A7FBBDE89D
:10339000FC8100000044004000080140103400207F
:1033A000102C0020800002403000002000000000AF
:1033B00000000000002F00000000070007000014BC
:1033C0007F147F1400242A7F2A12006264081323CA
:1033D00000364955225000000503000000001C2261
:1033E0004100000041221C000014083E081400089F
:1033F000083E0808000000A060000008080808084F
:10340000000060600000002010080402003E5149E6
:10341000453E0000427F4000004261514946002184
:1034200041454B31001814127F100027454545399E
:10343000003C4A49493000017109050300364949F9
:10344000493600064949291E0000363600000000B2
:1034500056360000000814224100001414141414FD
:1034600000004122140800020151090600324959A6
:10347000513E007C1211127C007F49494936003EC2
:1034800041414122007F4141221C007F494949417D
:10349000007F09090901003E4149497A007F080877
:1034A000087F0000417F4100002040413F01007F34
:1034B00008142241007F40404040007F020C027F00
:1034C000007F0408107F003E4141413E007F090912
:1034D0000906003E4151215E007F09192946004638
:1034E000494949310001017F0101003F4040403F0F
:1034F000001F2040201F003F4038403F0063140859
:103500001463000708700807006151494543000033
:103510007F41410000552A552A55000041417F0056
:10352000000402010204004040404040000001024B
:103530000400002054545478007F48444438003834
:103540004444442000384444487F003854545418BC
:1035500000087E0901020018A4A4A47C007F0804CE
:1035600004780000447D4000004080847D00007F9E
:10357000102844000000417F4000007C04180478BB
:10358000007C0804047800384444443800FC2424B7
:1035900024180018242418FC007C0804040800489F
:1035A0005454542000043F444020003C4040207CC0
:1035B000001C2040201C003C4030403C00442810AF
:1035C0002844001CA0A0A07C004464544C44141463
:1035D000141414140000000000000000000000009B
:1035E0000000FC000000000002000000000C020CC3
:1035F000020000000000000090D0BCD0BC9000038E
:10360000000300001824FE448C000302070201009E
:103610001824D8B04C80000300010201C038E438FF
:10362000E0000102020102020806000000000000A2
:1036300000000000000000F8040200000001020485
:10364000000204F800000004020100009060F8602D
:1036500090000000010000002020FC20200000005D
:10366000010000000000000000000806000000004B
:1036700020202020200000000000000000000000AA
:1036800000000002000000000080601C0200040333
:1036900000000000F8040404F80001020202010026
:1036A0000008FC000000000203020000188444240B
:1036B000180003020202020008042424D8000102B8
:1036C0000202010040B088FC8000000000030200FC
:1036D0003C242424C400010202020100F824242C0A
:1036E000C0000102020201000C04E41C04000000FE
:1036F00003000000D8242424D800010202020100A3
:1037000038444444F80000030202010000001000A5
:103710000000000002000000000020000000000087
:103720000600000000205088040200000000010292
:10373000909090909000000000000000000204882B
:1037400050200002010000001804C42418000000EA
:1037500002000000F804E494F800010202020200F2
:1037600000E09CF0800002030000030204FC24241B
:10377000D800020302020100F80404040C00010254
:103780000202010004FC0404F8000203020201002A
:1037900004FC24740C0002030202030004FC2474E1
:1037A0000C00020302000000F0080444CC400001B9
:1037B0000202010004FC2020FC04020300000302BA
:1037C0000404FC040400020203020200000404FCDE
:1037D000040406040403000004FC24D00C040203C7
:1037E0000200030204FC04000000020302020203C0
:1037F000FC3CC03CFC0003000300030004FC30C49C
:10380000FC04020302000300F8040404F8000102AF
:103810000202010004FC242418000203020000003C
:10382000F8848404F80001020207050004FC246403
:103830009800020302000302182424448C000302AF
:10384000020201000C04FC040C0000020302000050
:1038500004FC0000FC04000102020100047C80E082
:103860001C040000030000001CE03CE01C000003FE
:1038700000030000049C609C04000203000302009B
:10388000041CE01C04000002030200000C84641C01
:1038900004000203020203000000FE020200000016
:1038A00007040400000E30C0000000000001020008
:1038B000000202FE000000040407000000040204ED
:1038C00000000000000000000000000000000808E8
:1038D00008080808000002000000000000000000C6
:1038E0000040A0A0C00000010202030204FC20204E
:1038F000C00000030202010000C02020600000019F
:103900000202020000C02024FC00000102020302A7
:1039100000C0A0A0C0000001020202000020F824A4
:1039200024040002030202000040A0A0602000075F
:103930000A0A0A0404FC2020C00002030200030259
:103940000020E4000000000203020000000020E468
:10395000000008080807000004FC80E020200203A3
:10396000020003020404FC00000002020302020041
:10397000E020E020C00003000300030020E020203E
:10398000C00002030200030200C02020C0000001AA
:103990000202010020E02020C000080F0A020100FE
:1039A00000C02020E0000001020A0F0820E04020B3
:1039B00020000203020000000060A0A0200000021E
:1039C000020203000020F8200000000001020200B3
:1039D00020E00020E00000010202030220E020803D
:1039E00060200000030100006080E08060000003B0
:1039F000000300002060806020000203000302003A
:103A000020E0208060200808070100000020A0605E
:103A10002000000203020200000020DE020000007D
:103A200000070400000000FF00000000000F00007D
:103A30000002DE2000000004070000000201020472
:103A40000402000000000000000000000000000070
:103A50000000000000000000000000F8000000006E
:103A6000000000333000000000100C06100C0600AF
:103A7000000000000000000040C07840C078400016
:103A8000043F04043F040400007088FC0830000078
:103A9000001820FF211E0000F008F000E0180000D0
:103AA00000211C031E211E0000F008887000000089
:103AB0001E2123241927211010160E0000000000DB
:103AC0000000000000000000000000E018040200F8
:103AD000000000071820400000020418E000000069
:103AE0000040201807000000404080F08040400067
:103AF0000202010F01020200000000F000000000BD
:103B00000101011F01010100000000000000000090
:103B100080B0700000000000000000000000000005
:103B2000000101010101010100000000000000008E
:103B30000030300000000000000000008060180429
:103B4000006018060100000000E010080810E00006
:103B5000000F102020100F00001010F800000000CF
:103B60000020203F20200000007008080888700016
:103B70000030282422213000003008888848300096
:103B80000018202020110E000000C02010F80000B6
:103B900000070424243F240000F80888880808004F
:103BA0000019212020110E0000E010888818000064
:103BB000000F112020110E0000380808C838080036
:103BC0000000003F000000000070880808887000B6
:103BD000001C222121221C0000E010080810E00037
:103BE0000000312222110F00000000C0C0000000C0
:103BF00000000030300000000000008000000000E5
:103C000000008060000000000000804020100800DC
:103C100000010204081020004040404040404000A5
:103C20000404040404040400000810204080000080
:103C30000020100804020100007048080808F00085
:103C40000000003036010000C030C828E810E00055
:103C50000718272423140B000000C038E0000000E0
:103C6000203C23020227382008F88888887000004A
:103C7000203F202020110E00C0300808080838001E
:103C8000071820202010080008F808080810E00095
:103C9000203F202020100F0008F88888E808100036
:103CA000203F20202320180008F88888E80810000A
:103CB000203F200003000000C03008080838000042
:103CC00007182020221E020008F808000008F80843
:103CD000203F210101213F20000808F808080000CA
:103CE0000020203F2020000000000808F8080800FD
:103CF000C08080807F00000008F888C02818080075
:103D0000203F20012638200008F8080000000000AD
:103D1000203F20202020300008F8F800F8F80800A4
:103D2000203F003F003F200008F830C00008F8089E
:103D3000203F200007183F00E01008080810E000AE
:103D40000F10202020100F0008F808080808F000C5
:103D5000203F210101010000E01008080810E000E8
:103D60000F18242438504F0008F88888888870007D
:103D7000203F2000030C302000708808080838001D
:103D80000038202121221C00180808F80808180013
:103D90000000203F2000000008F808000008F80894
:103DA000001F202020201F000878880000C8380845
:103DB000000007380E010000F80800F80008F800BD
:103DC000033C0700073C0300081868808068180857
:103DD00020302C03032C30200838C800C8380800D5
:103DE0000000203F2000000010080808C838080024
:103DF0002038262120201800000000FE02020200C8
:103E00000000007F40404000000C30C00000000077
:103E1000000000010638C00000020202FE0000009F
:103E2000004040407F000000000004020202040045
:103E30000000000000000000000000000000000082
:103E4000808080808080808000020204000000006A
:103E50000000000000000000000080808080000062
:103E60000019242222223F2008F800808000000050
:103E7000003F112020110E00000000808080000013
:103E8000000E112020201100000000808088F80022
:103E9000000E112020103F20000080808080000054
:103EA000001F222222221300008080F088888818B8
:103EB0000020203F202000000000808080808000C3
:103EC000006B94949493600008F800808080000058
:103ED000203F210000203F20008098980000000033
:103EE0000020203F20200000000000809898000063
:103EF00000C08080807F000008F800008080800083
:103F0000203F24022D302000000808F800000000A7
:103F10000020203F20200000808080808080800062
:103F2000203F20003F20003F8080008080800000F4
:103F3000203F210000203F20000080808080000082
:103F4000001F202020201F008080008080000000B3
:103F500080FFA12020110E000000008080808000E2
:103F6000000E112020A0FF808080800080808000D3
:103F700020203F2120000100000080808080800000
:103F80000033242424241900008080E08080000075
:103F90000000001F202000008080000000808000C2
:103FA000001F202020103F20808080000080808023
:103FB00000010E30080601008080008000808080B3
:103FC0000F300C030C300F000080800080808000D8
:103FD0000020312E0E312000808080000080808003
:103FE00080818E70180601000080808080808000B3
:103FF0000021302C2221300000000000807C0202D1
:1040000000000000003F404000000000FF000000F2
:1040100000000000FF0000000002027C80000000A1
:104020000040403F000000000006010102020404BD
:104030000000000000000000000000000000000080
:104040000000000000000000000000000000000070
:104050000000000000000000000000000000000060
:1040600000F0F0F0000000000000000000017F01FF
:104070000000000000000000001C1C1C00000000EC
:1040800000008060301C8C60301C0C0000000000C0
:104090000000000000000000000000000000000020
:1040A00000000000000000E00000000000E0000050
:1040B0000086E69F86868686E69F860000011F01B1
:1040C000010101011F010100000080C06020F820F3
:1040D000E0C00000000003070C18FF70E181000041
:1040E0000000070F10107F100F0700008060206095
:1040F00080000000E02000000F3020309F70DC378F
:104100001030C0000000100E030007181018070040
:104110000000C02020E0C0000000000080E01F3848
:10412000E88703C43C040000070F1810100B070DAC
:104130001010080000808C4C3800000000000000C7
:10414000000000000000000000000000000000006F
:10415000000000000000000000000000000080E0FF
:10416000300804000000000000FEFF010000000015
:10417000000000000000030F182040000004083079
:10418000E0800000000000000000000001FFFE00D1
:1041900000000000004020180F0300000000000095
:1041A000000000000000C000000000000042666641
:1041B0003C18FF183C666642000000000000030047
:1041C000000000000000000000008000000000006F
:1041D000001010101010FF10101010100000000040
:1041E00000000300000000000000000000000000CC
:1041F00000000000000000000000000000000000BF
:1042000000808C4C3800000000000000000000001E
:10421000000000000000000000101010101010102E
:10422000101010000000000000000000000000005E
:10423000000000000000000000000000000000007E
:10424000000000000000000000001C1C1C0000001A
:10425000000000000000000000000000E0380C003A
:104260000000000080701C03000000000060380E99
:104270000100000000000000000080C060202060FD
:10428000C080000000FEFF010000000001FFFE00F2
:104290000001070E181010180E07010000008080A2
:1042A00080C0E000000000000000000000FFFF00F0
:1042B0000000000000001010101F1F101010000060
:1042C0000080402020202060C08000000003030008
:1042D000804020381F070000001C1A1918181818F1
:1042E000181F00000080C020202060C08000000057
:1042F000000303001010182FE780000000070F10C4
:10430000101010180F070000000000000000C0E0AF
:10431000F000000000C0B088868180FFFF80800030
:10432000000000000010101F1F1010000000E060CF
:10433000606060606060000000003F1008080818BE
:10434000F0E0000000070B101010101C0F0300001D
:10435000000080C040202020E0C0000000FCFF21C1
:104360001008080818F0E0000001070C18101010E1
:10437000080F03000000C0E06060606060E0600063
:10438000000003000000E01807000000000000002B
:10439000001F1F00000000000080C06020202020BF
:1043A00060C080000087EF2C1818303068CF830081
:1043B00000070F0810101010180F07000000C0C0F1
:1043C00020202020C0800000001F3F60404040208F
:1043D00010FFFE0000000C1C101010080F0300005E
:1043E00000000000000000000000000000000000CD
:1043F000000E0E0E0000000000000000001C1C1C3F
:1044000000000000000000000000000000000000AC
:1044100000000000000C0C00000000000000000084
:10442000005838000000000000000000000000807C
:10443000402010000000102844820100000000000D
:10444000000000000000010204081000000000004D
:1044500000000000000000000084848484848484C0
:1044600084848400000000000000000000000000C0
:10447000000010204080000000000000000000004C
:10448000000001824428100000001008040201000E
:104490000000000000C020201010101030E0C0000C
:1044A0000003030000F010080C07030000000000E8
:1044B0001C1C1C0000000000000000C04060202008
:1044C0002040C00000FCFF01F00E03C1FE03807F0E
:1044D0000001070E0811111011090402000000006C
:1044E00080E0E000000000000000807C4340477F47
:1044F000F880000010181F1000000000131F1C108F
:1045000020E0E02020202060C080000000FFFF109D
:10451000101010182FE78000101F1F10101010101F
:10452000180F0700000080C0402020202060E0001D
:1045300000FCFF0100000000000001000001070E68
:10454000181010100804030020E0E0202020204074
:10455000C080000000FFFF000000000001FFFE001F
:10456000101F1F10101018080E07010020E0E02097
:10457000202020202060800000FFFF101010107C01
:1045800000000000101F1F1010101010101806005F
:1045900020E0E020202020206060800000FFFF104D
:1045A0001010107C00000100101F1F100000000000
:1045B00000000000000080C06020202040E00000DB
:1045C00000FCFF0100004040C0C140400001070E58
:1045D000181010100F0F000020E0E0200000000075
:1045E00020E0E02000FFFF101010101010FFFF006F
:1045F000101F1F1000000000101F1F1000002020BF
:1046000020E0E020202000000000000000FFFF006C
:104610000000000000001010101F1F1010100000FC
:1046200000000000202020E0E0202020000000000A
:10463000000000FFFF0000000060E0808080C07F7D
:104640003F00000020E0E020000020A060202000CB
:1046500000FFFF30187CE3C000000000101F1F1097
:10466000000001131F1C181020E0E02000000000D3
:104670000000000000FFFF0000000000000000003C
:10468000101F1F10101010101018060020E0E0E09E
:1046900000000000E0E0E02000FF013FFEC0E01E5F
:1046A00001FFFF00101F1000031F0300101F1F1049
:1046B00020E0E0C0000000000020E02000FF000338
:1046C000071C78E08000FF00101F100000000000B1
:1046D000030F1F00000080C060202060C080000029
:1046E00000FEFF010000000000FFFE000001070EB9
:1046F000181010180C07010020E0E02020202020D6
:1047000060C0800000FFFF2020202020301F0F000D
:10471000101F1F100000000000000000000080C0FB
:1047200060202060C080000000FEFF01000000004B
:1047300000FFFE000001070E1111133C7C672100F1
:1047400020E0E0202020202060C0800000FFFF103B
:104750001030F0D0080F0700101F1F1000000003DA
:104760000F1C10100080C060202020204040E0007E
:1047700000070F0C1818303060E08100001F0C0893
:1047800010101010180F07008060202020E0E0209B
:10479000202060800100000000FFFF0000000001F9
:1047A00000000000101F1F100000000020E0E020AB
:1047B000000000000020E02000FFFF0000000000DB
:1047C0000000FF0000070F1810101010100807005D
:1047D0002060E0E02000000020E060200000077F73
:1047E000F88000807C03000000000000071F1C0709
:1047F0000000000020E0E02000E0E0200020E020B9
:104800000007FFF8E01FFFFCE01F00000000031F8F
:104810000300011F03000000002060E0A000002052
:10482000E0602000000000038F7CF8C6010000005B
:104830000010181E130001171F1810002060E0E080
:104840002000000020E06020000001073EF8E01892
:104850000700000000000010101F1F1010000000D3
:1048600000806020202020A0E0E020000000000068
:10487000C0F03E0F0300000000101C1F17101010A6
:10488000101806000000000000FC040404040400EA
:104890000000000000FF0000000000000000000019
:1048A000007F404040404000000010E00000000059
:1048B0000000000000000000031C608000000000F9
:1048C00000000000000000030C70800000000404E1
:1048D000040404FC0000000000000000000000FFD1
:1048E00000000000000040404040407F0000000009
:1048F00000000010080C040C08100000000000006C
:1049000000000000000000000000000000000000A7
:104910000000000000000000000000000000000097
:104920000000000000000000000000008080808087
:10493000808080808080808000000004040808005F
:104940000000000000000000000000000000000067
:104950000000000000000000000000000000000057
:104960000000000000000000000098D844642424E7
:10497000FCF80000000F1F18101010081F1F10185F
:104980000020E0F000000000000000000000FFFF39
:10499000180804040CF8F00000001F0F1810101085
:1049A000180F0300000000000000000000000000DD
:1049B00000E0F8180404043C3800000000030F0C69
:1049C0001010101008060000000000000000002079
:1049D000E0F0000000E0F81C04040408FFFF000001
:1049E00000030F18101010081F0F0800000000002F
:1049F00000000000000000000000E0F848444444CB
:104A00004C7870000000030F0C1810101008040000
:104A10000000000080C0602020E0C000000404040A
:104A2000FFFF040404040000000010101F1F1010FA
:104A30001000000000000000000000000000000066
:104A4000000070F88C04048CF874040C007076CFAD
:104A50008D8D8D89C87870000020E0F00000000086
:104A6000000000000000FFFF08040404FCF8000040
:104A700000101F1F100000101F1F1000000000007A
:104A800000606000000000000000040404FCFC0062
:104A90000000000000001010101F1F101010000078
:104AA0000000000000000060600000000000000046
:104AB000040404FCFC0000000000C0C08080C07F33
:104AC0003F0000000020E0F00000000000000000B7
:104AD0000000FFFF80C0F41C0404000000101F1F32
:104AE0001100031F1C1010000000202020E0F00027
:104AF000000000000000000000FFFF0000000000B8
:104B000000001010101F1F10101000000000000007
:104B1000000000000000000004FCFC0804FCFC088D
:104B200004FCFC00101F1F10001F1F10001F1F108F
:104B30000000000000000000000000000004FCFC79
:104B400008080404FCF8000000101F1F10000010EB
:104B50001F1F100000000000000000000000000007
:104B600000E0F0180C04040C18F0E00000030F0C37
:104B7000101010100C0F03000000000000000000D7
:104B8000000000000004FCFC080404040CF8F00021
:104B90000080FFFF889010101C0F03000000000031
:104BA000000000000000000000E0F81C04040408FD
:104BB000F8FC000000030F1810109088FFFF800021
:104BC000000000000000000000000000040404FCDD
:104BD000FC100804040C0C001010101F1F10101003
:104BE00000000000000000000000000000000000C5
:104BF00000003078CCC48484840C1C0000001E1893
:104C000010101011190F06000000000000C0000075
:104C10000000000000040404FFFF0404040000007E
:104C2000000000000F1F1010100C0000000000001A
:104C300000000000000000000004FCFE0000000472
:104C4000FCFE000000000F1F181010081F0F0800C6
:104C500000000000000000000000000000040C3C08
:104C6000FCC40000C43C0C0400000000010F1E0E38
:104C70000100000000000000000000000000000033
:104C8000043CFCC400E47CFC84807C040000071F1E
:104C9000070000071F0700000000000000000000E0
:104CA000000000000004041C7CE4C0341C04040068
:104CB0000010101C1601131F1C181000000000002B
:104CC000000000000000000000040C3CFCC400C414
:104CD0003C0404000000C080C1370E010000000049
:104CE00000000000000000000000000000001C04A4
:104CF00004C4F47C1C0400000000101C1F171110D9
:104D000010180E0000000000000000F80C04000065
:104D100000000000001028EF00000000000000006C
:104D20000000003F60400000000000000000FF00A5
:104D300000000000000000000000FF000000000074
:104D4000000000000000FF00000000000000040C54
:104D5000F80000000000000000000000EF28100034
:104D600000000000000040603F0000000000000064
:104D7000001806020204081020203008000000007D
:104D80000000000000000000000000000000000023
:104D9000000000000000800000E002041800000095
:104DA00040800000100C0300003F4040404040782D
:104DB00000010E000014A4442434AD66249404447D
:104DC000A414000008090808090909FD09090B08CD
:104DD000080908000000F80808F80C0B08F8080893
:104DE000F800000040407F40407F4040407F40400E
:104DF0007F4040000824236AAA2AAA6A2A2A2AEAAB
:104E0000020200001011151515FF15151511100FD0
:104E10003040F800000000C080808080808080FCEE
:104E200084808080808080C0C0000000000000FF7F
:104E30007F404040404040FF40404040404040FFB5
:104E40007F00000000000000000000000000007F64
:104E500070000000000000000000000000000000E2
:104E60000000000000000000000000FCF80000004E
:104E70000000000000000000000000000000000032
:104E8000FFFE020202020202020202FFFF0202020F
:104E9000020202020202FF03000000000000000004
:104EA0001F1F040404040404040404FFFF04040496
:104EB0000404040404041F000000000000000000BB
:104EC00000000000000000000000007F3F00000024
:104ED00000000000000000000000000000000000D2
:104EE00000000000000000000000000000000000C2
:104EF000000000000000000000F8F8F0F070200052
:104F000000000000000000000000000000000000A1
:104F10000000000000000000000000000000000091
:104F20000000000080000000000000000000000001
:104F3000000000000000000000FFFFFFFF00000075
:104F40000000000000000000000000000000000061
:104F50008080000000000000000000000000000051
:104F60000000000000FFFFFE060606060606060615
:104F7000060606060606060606FFFFFFFF060606ED
:104F8000060606060606060606060606060606FFC8
:104F9000FFFFFF070200000000000000000000000B
:104FA0000000000000FFFFFF000000000000000004
:104FB000000000000000000000FFFFFFFF000000F5
:104FC000000000000000000000000000000000FFE2
:104FD000FFFFFF00000000000000000000000000D4
:104FE0000000000000FFFFFF181818181818181804
:104FF000181818181818181818FFFFFFFF18181895
:10500000181818181818181818181818181818FF39
:10501000FFFFFF0000000000000000000000000093
:10502000000000000201010000000000000000007C
:10503000000000000000000000FFFFFFFF00000074
:10504000000000000000000000000000000000015F
:10505000010000000000000000000000000000004F
:105060000000000000000000000000000000000040
:10507000000000000000000000FFFFFFFF00000034
:105080000000000000000000000000000000000020
:105090000000000000000000000000000000000010
:1050A0000000000000000000000000000000000000
:1050B0000000000000000000001F1F0F0F00000094
:1050C00000000000000000000000000000000000E0
:1050D0000000000000000000000000002900140192
:1050E0000002140129000000000000000000000080
:1050F00000000000000000000000000000000000B0
:10510000000000000000000000000000000000009F
:10511000000000000000000000005F5F5F60606052
:10512000616161616162626262626363636363635E
:105130006363646464646464646464646464646431
:10514000646464646464636363636363636362622B
:105150006262626261616161606060605F5F5F5E48
:105160005E5E5D5D5D5C5C5C5B5B5A5A595959588B
:1051700058575756565555545453525251515050F2
:105180004F4E4E4D4C4C4B4A4A4948484746454580
:105190004443424241403F3E3E3D3C3B3A39383831
:1051A00037363534333231302F2E2D2C2B2A292807
:1051B000272625242322211F1E1D1C1B1A19171602
:1051C00015141311100F0E0C0B0A09070605030224
:1051D00001000000F4510008000000205000000011
:1051E000641F00084452000850000020D03700001F
:1051F000741F000800000000000000000000000014
:10520000000000000000000000000000000000009E
:10521000000000000000000000000000000000008E
:10522000000000000000000000000204060800006A
:10523000000001020304010203040607080900003C
:04524000000000006A
:04000005080000ED02
:00000001FF
